:020000022000DC
:1000000000C0FF24F8BE0091780005FD0AC1F092FF
:10001000A00608E10093B5060FEF0A950023E9F763
:100020000091A80600FFEAC0E0E0F0E00791169119
:100030000F3F19F41F3F09F4E1C0F3C027E402EABF
:1000400010E00F94FF000F947D0378940F946304E5
:100050000F94F308FFCF3BB72BBFF8012091CA01E3
:100060004093CA013DE930933400E8952093CA01DA
:100070003BBF08953091CF0137FDFCCF3BB72BBF7D
:10008000F8012091CA0113E21093CA010A01E89510
:080090002093CA013BBF089553
:1001F4000D9420090D94570907C040E04BBFF80146
:1002040058ED54BF2083089501E70DBF00E20EBFEF
:10021400CAEADAE2E0E0EABF0F94B90B0DDFF0922C
:10022400B50600910020109101200A3A154511F0FD
:100234000C940000F0920020F092012000E2009360
:100244007800F6CF4091CA01E22FF32F0093CA0140
:1002540004914093CA0108954A951AF0000F111FA2
:10026400FBCF08954A951AF016950795FBCF08958C
:10027400AF93BF93D8013BBF29BF01900D9241506A
:1002840050406040D1F7BF91AF910895FA92EA923D
:10029400DA92CA92BA92AA929A928A927A926A92BA
:1002A4005A924A92BA93AA939A938A930895FF848E
:1002B400EE84DD84CC84BB84AA84998488847F8082
:1002C4006E805D804C80BB81AA8199818881F0E039
:1002D400EC0FFD1FEF0108950A011B01B901A801EC
:1002E400800191010D94A602E1E0EA930D94C70206
:1002F4000A01A901980180010D94D1019A01AB0171
:100304000D9404020A01A90122E730E2200D311DF7
:100314000D948B0B0A01A90120E531E2F7CF00917E
:10032400900000935021009191000093512100917D
:100334009200009352210091930000935321089559
:10034400E0EDF1E030E03BBF008101FB00E000F9AB
:100354000F27089530E00091CF0107FDFCCF40E264
:1003640000E010E020E00F942B000F949F0201E0C6
:100374000895F8940AEA15E50093002010930120EB
:1003840020917900216009E710E00F94FF00FFCF6E
:100394000895E4E00D94650130E03BBF0895B80191
:1003A400890192D03BBF208127FDFCCFECEC20815A
:1003B40028602083705F9B010F948B0BECECF1E0C1
:1003C40030E057D0077F008308950F945401C8018B
:1003D400A22FB091CA013DD077D04BD007FDFDCFFD
:1003E4000DD03093C2019093C1018093C001A093BA
:1003F400C40105E338D0B093CA01CBCF03E3009323
:10040400CA0108950F945201C8012901DA010BC0F1
:10041400820135D045E08C010F9434014DD0809693
:1004240000E2AFD090970A2F0B2B81F0082F0F71A9
:1004340021F4A03200E0B00758F7F201ADDF2191BA
:100444002F018C01C2DF01961197EDCFE6E00D94E8
:1004540063013AD00ED007FDFDCF008101FF02C039
:1004640006E301D00895CBDF21E00BEC11E00D94FD
:10047400FF003BBF008108954093CA010895409155
:10048400CA0130E02091CF0127FDFCCF23E3209364
:10049400CA0120E00CD02093C001F8013BBF519168
:1004A4008F015093C40123952032A8F3E5CF3093F4
:1004B400C2013093C101089506D035D017FDFDCF98
:1004C40007D005E32AC08A93EFECF1E030E0089509
:1004D40010E045E00F942E013093C2011093C10146
:1004E4000093C0018091CA0108959A938A93802F42
:1004F4009091CA01AEDF30E0BBD007FDFDCF7EDFB7
:1005040000E0D5DF1ED08093C40103950032D0F300
:100514009093CA0189919991089571DFA5DF809321
:10052400CA01899108953BBF10810895CCDFA1DFF2
:1005340007FDFDCFD7DF00E3F0CF01D0F7CF0FEFFA
:10054400D4CF0093C00108951C0108018A01CB0196
:10055400A001622F30E02091CF0127FDFCCF282F8E
:10056400292B61F0FA016BBF2691F8013BBF21935F
:100574008F014F5F5F4F6F4F0197F1CFC101089516
:1005840001E0400E00E0501E08950F9448012297A8
:100594007A014B01AA88280139011170802F952D09
:1005A400D901801B910BA040B04007C061D007FD6A
:1005B400FDCF45E2002D0F942B00082D092909F4E5
:1005C40053C0BB2455D007FDFDCFCC24DD24D394E8
:1005D400AA2071F0FC01ABBF07911691088319831F
:1005E4004881512F4F3F5F4F31F0BB24B39403C078
:1005F4000FEF08830983082D0929B9F04816590615
:100604006A067B0629F437D00883082D092969F086
:100614008C019D010F5F1F4F2F4F3F4F4016510616
:100624006206730611F427D00983488159818C012D
:100634009D010F943A008E5F9F4FAF4FBF4F0FEF56
:10064400C00ED01E0C2D0D2919F68C019D010050F1
:10065400124020403040BB20002E09F0A7CF08D024
:1006640007FDFDCF44E2A6CF2296E1E10D945901A6
:100674000091CF0108950FEF800E901E81DF601E60
:10068400701EF7010BBF01917F0108953FB7F894E5
:100694000A9519F00A9559F027C01830E6E550D0AC
:1006A40011F4016001C00E7F0083E8E61AC0E6E59C
:1006B40047D0097F0083183021F400810260008351
:1006C4000FC01F3F21F412D000810460F8CF143012
:1006D40039F40CD039D0008104602ED00681068311
:1006E400E0E60081016000833FBF089500E80787CA
:1006F4000BEB008B08952497E0E7F0E007E01FEF91
:1007040030E03BBF11930A95E1F724E001E410E0E7
:100714004FD02CE130E051D012D00DD0E1E5008172
:1007240001FFFDCF21E000E442D044D008D00E7F89
:1007340003D024960895026000831FBF089504D057
:10074400F0E0FBBF008108951FB7F894E0E5089539
:100754002FB7F894109504D0012300832FBF089578
:10076400F0E0E02FE059FF4F30E03BBFEBCF8A933E
:100774002497063011F488E101C080E00091510013
:1007840001FB5EF0E1DFF0E0EFDFD5DF0091510027
:1007940001FBE6F72CE111D00DD08360282F04E48F
:1007A40006D010E400E0D4DF24968991089510E087
:1007B4000D94FF001FEF02E069CF18D009832DE1EB
:1007C40030E014D0088319810F3F1F4F21F400E457
:1007D40013E208831983088119810A831B830A8120
:1007E400009362000B8100936300089502E00D946E
:1007F40024010F94540159D12681222311F400E0DD
:1008040032C0A281B38190E039BF4D915C91DA018D
:10081400149639BF2C91021790F744835583DA015B
:1008240012962D913C91420F531F07C06C91048086
:100834001580060E191E04821582A481B581A417A1
:10084400B507E8F6119699BF2C911197243071F7EA
:1008540012962C911297021749F713962C9113971D
:10086400121721F701E0E4E00D9465018A93802FCB
:1008740010E052D111F400E006C016D003811481B7
:100884002581E8D101E0899108958A93802F44D18C
:1008940049F00AD0008111812281DCD1002311F0BA
:1008A40001E001C000E0EFCFE0915621F091572123
:1008B400A8D1D8D1829FF6D0F8010081F181E02F30
:1008C40008950D94B908AA931CD131F0A0E002C098
:1008D40039D1A395CBD1E0F300E000935A2101E094
:1008E40010E092D11BBF00831183A99108958A93CC
:1008F40008D1D9F080E00FC0F801B4D1829F90D024
:1009040004841584268403161306230619F0F001C3
:100914002CBE199583950091562110915721F80109
:1009240070D180D02481821738F3ADCF0091E429AF
:100934000F770D9411090091E429002329F00A95F9
:1009440041F00A9519F126C024E030E006E011E2F6
:100954001BC025E00EEE10E240E050E032E0F8016A
:10096400E40FF51F5BBF6081439FF001E653FF4D29
:10097400628353834395421790F3220F2E5F209393
:10098400CA2030E00AEC10E2BAD005C021E104EF3D
:1009940010E2E2CF02C001E0089500E00895BA93A6
:1009A400AA93A2EEB9E22CD16281238104E411E27C
:1009B4002A9529F02A9559F02A9511F10CC0F801CD
:1009C40040815181FA0120818A0199D01CC029D02B
:1009D4002189621710F000E020C0F8010281138120
:1009E40024E0629F1DD022813381F801042F1181FC
:1009F40086D022E005D10085F185E02F218303C054
:100A04009ADF002341F3FD0128D142855385041761
:100A1400150710F40287138701E0A991B99108958D
:100A240041D0F8014081F181E42F08959A938A938B
:100A340082EE99E2FC0188D021F000E0899199913D
:100A440008950F9414090023C1F3E0914421F09117
:100A54004521D7D02189FC010281201770F333DFAF
:100A6400FC01CFD0028100935A2120915A212223E4
:100A740011F401E0E3CF009146211091472134E0C5
:100A8400239F10D004501040BFD00283138380E012
:100A94000CD03BD070F710E0082FF7DE002369F28A
:100AA4008395F6CF000D111D0895E4E5F1E2A9C088
:100AB4000F9454010091E8291091E929013020E0B4
:100AC400104011F000E01AC0A4E5B1E21AD0D1F34D
:100AD4008091E629FD012BBF18D0A0F710E0082F64
:100AE4001BD081F3FD01BDD0E5DEB1D000935B21C5
:100AF40021E030E017968D0102D001E0B4CE0D94D0
:100B0400170900915A21002308950281F381E02FEF
:100B1400B3D0801708950A2F6CDEF5CFAA938A9379
:100B2400E2EEF9E211D011F000E00AC0EADFE1F3ED
:100B3400A481828107D00023B9F3182F0A2FA5DEE0
:100B44008991D3CE0A2F92CE88D0012B0895E2EE5C
:100B5400F9E257D0008107FF2AC046815781042F4C
:100B6400052B99F100810F71E1F41181112329F012
:100B7400165061F0125059F014C0423000E0504059
:100B840009F0089522E004E511E209C008CF4130DC
:100B940000E0504009F0089521E00AE511E2AFDFDA
:100BA400FACE013091F401810A3079F481CF0F71CA
:100BB40009F511811A9589F0125039F0125019F083
:100BC4001450B9F017C084D009F0E7CE08E914E056
:100BD40021E0048715872687E3CF7AD0B1F7028115
:100BE40013810130104089F70FD000810D7F0083FD
:100BF400D7CF1CCF013049F701810B3031F78ECFAD
:100C0400FD0130E03BBF0895E4E5F1E208950F945F
:100C1400550177DF11F400E017C0A091E62926D032
:100C2400D0F710E078DFB9F3EFDF1BD0A29F3ADFF3
:100C3400F80180819181FC010AD0102F6CDF59F3F7
:100C4400FC010BD0208506D0E3E00D9466010185FC
:100C540012852385F8012CBF1994D3DF06811781EF
:100C640008950FD00281138122E00895E4E5F1E2B2
:100C740008D002D0A01708950081F181E02F0481EB
:100C84000895BFDF0281F3811ACEE2EEF9E200E0BB
:100C94000BBF028703870487058706870787008BB6
:100CA400018B008107FF03C013D009F476CE0091B5
:100CB400E229007621F44BDF002309F06CCE009189
:100CC400E2290F71013091F7A2DF0023B9F7EECFCB
:100CD400068117813ACF00E00093772158D00F9412
:100CE40091010F94A201DFC0089529D1A2EEB9E2C7
:100CF4000091E2290076003209F047C01091E329FF
:100D040090E099BF0C9107FF18C0125049F01A9552
:100D1400C1F526E030E006E611E279D101E036C003
:100D24007AD09BBF408D518D628D40305907690741
:100D340041F1FA016CBF199529C01A9521F013509D
:100D440001F525D0EBCF00917721002361F000E07D
:100D54000F94CA010BEB11E021E0FD019BBF048756
:100D640015872687DBCF20E430E00AE711E24FD174
:100D740009ED16E021E0FD019BBF0787108B218B55
:100D8400CDCF49D00FE09BBF69D000E091C102C034
:100D940000E0089500E0F8D0E2EEF9E200E00BBFD5
:100DA4000787008B018B0487058706870895EFDF8B
:100DB40000E031D00BBF008F018F028F01E00F9450
:100DC400CA01EAE7F1E226D150814181403001E0D5
:100DD400500709F423C0403003E0500709F441C030
:100DE4004130500709F457C0403004E0500739F44B
:100DF4000F94AC01002300E009F4089554C043307B
:100E0400500721F401E000937721089543305640C0
:100E140009F455C0BDCFECE5F1E20895FAD0048D94
:100E2400158D012309F0ADC047815085618540309F
:100E34005040604011F411D002C028D009F4A8CF6A
:100E440020E038E0E2D004E818E021E0E2EEF9E244
:100E5400E1D00787108B218B28C003E002870AE0CA
:100E6400A4CF14D019F023D011F4F7DF91CF048D5F
:100E7400158D012321F003EC17E021E003C00CEFF2
:100E840017E021E0008F118F228F0FC00CE711E2D1
:100E940081D000230895FADF19F009D011F4DDDFC1
:100EA40077CFBBD002C00093782101E00895B1D080
:100EB40044815581668140305040604008953FD060
:100EC400249700917D2110917C21112319F01A950A
:100ED400A9F032C0013140F008E0009366210AE035
:100EE40000936A2100E029C02CD000E0ACE6B1E216
:100EF40009BF0D930D930D930C931EC040E04883DE
:100F040049834A834B830B8300917E210A83ACE59A
:100F1400B1E248815981602F7B8190E099BF0D91A6
:100F24001D912D913C911397401751076207730748
:100F340098F6FD019BBFC9D001E02496B9C00D9479
:100F44005401033041F0023031F0043021F0053017
:100F540011F011E001C010E01093792112E0019F1B
:100F6400F001E955FF4D56D00080F1810CE511E206
:100F740020E0E02D4AE050E060E00D943A01FD01EC
:100F840049C003E001D004CF0093662102E000933E
:100F94006A2108950F945001ACE5B1E2F0DF628953
:100FA4007389F8011080512D0180402DFD01008AC4
:100FB400118A628B738B1B01F80112800380FD017F
:100FC4004080518062807380041415042604370421
:100FD40020F008E043DF00E00AC0041A150A260ADC
:100FE400370A01E0000E131E231E331E69D0E8E009
:100FF4000D9461010ED0248835896FD0222D6AD0DA
:1010040008D02489358901D050CF0AEB11E20D9420
:10101400170901DF30E03BBF089594D04CD0452B35
:10102400462B472B41F458EF348B558B368B378B3B
:1010340080E098E019C0A3DF3ED0042F052B062BD7
:10104400072BB1F1403008E050076040704010F4C5
:10105400CA0102C080E098E00A0126883788081A8D
:10106400190A230A330A2CD0392F37D0282F32D02B
:101074000AEB11E208C0FD013BBF36D04F5F5F4F62
:101084006F4F7F4F22D09C010197232BA1F2F801CF
:10109400C1DF21918F012F3F71F305E00093662199
:1010A4000BE718E021E0FD013BBF008F118F228F79
:1010B400E4E00D946501448955896689778908952A
:1010C400048A158A268A378A0895408B518B628B4D
:1010D400738B08950AEB11E2199406D004811581EB
:1010E4002681F8012CBF089540895189628973894A
:1010F40008958FDF408901890093BA214093BB2171
:1011040022E081CF1FD00088118822893389648925
:101114007589002D0F7310E04AEB51E2400F511F07
:10112400800190E0179699BF0D901D902C90F001CE
:101134002CBE1995E2EEF9E29BBF9787908B918BB9
:1011440001E0B6CFFCDEACE5B1E219CF2AE107D06D
:101154000093FA042BE103D00093FB04089530E0DC
:1011640002E00F9424010F3F09F40FE108958A93DC
:1011740000E00093600000E30F94B90385D100649C
:10118400008301E0009360000FB7F894802F20E003
:10119400890107D1F801E054F64D318B23952230B3
:1011A400B8F3D4DF0091C0040093C0046DD100688B
:1011B4000083008100611BD17096E093C604F09314
:1011C400C704E0ECF4E00081006200830FEF0583C4
:1011D400E8EC0081016000838FBF8991089500E0ED
:1011E40008951FB7F89400E47DD200E27BD2E1ECCD
:1011F4004CD101600083E9EC008102600083E8ECDB
:10120400008100640083E9EC008101600083E8EC64
:101214000081006800831FBF089500830895009330
:10122400C30408950091C30408950093EA29109318
:10123400EB292093EC293093ED2908956FD000E039
:1012440008BF0091CB0407FF05C000E84BD20F9400
:10125400790429C030D2002331F5EBEC16D104FF18
:1012640018C000E13FD20F94650400E00093C3046A
:1012740020E430E010E06BD020E430E010E000E83F
:1012840066D00AEF19E20093D4291093D52961D1CD
:101294000AC0008106FF02C000E404C0008105FF0B
:1012A40002C000E21FD21BD0189538D000E008BF5E
:1012B4001CD2002399F402E00093CC040091C504ED
:1012C40000E02BD0F801BED1008105FF04C000E08E
:1012D4001FD040D103C000E81BD0DCD0E4CF4CBE0B
:1012E400BBBFA9BF98BF8FBF0991199129913991AB
:1012F400499159916991799109901990299039905E
:10130400E991F99189919991A991B9914990089597
:1013140004D0F801BBD00F7D80CF34C04A92BA9379
:10132400AA939A938A93FA93EA933A922A921A92F4
:101334000A927A936A935A934A933A932A931A9302
:101344000A938FB798B7A9B7BBB74CB608958A93D9
:101354002051304041F02051304039F0205230408B
:1013640031F080E005C081E003C082E001C083E089
:10137400D4DF20E0F8012BBF218326E020838064A2
:1013840081832BCF60ED79E2202F2F70220F402F25
:10139400440F00E010E0001F020F03D0060F171FD8
:1013A400089543E00D942E01E8ECF4E0B3DF0081EE
:1013B4000F7D1DD0008D0260008F328F338F008D22
:1013C4000F7D008F008D0F7B008F00890F7D008BB8
:1013D40000890F7B008BE2EEF9E23487358736878C
:1013E4003787308B318B32873387368B0895008370
:1013F400E0ECF9E20895A5D0002331F0033011F0B8
:10140400043009F449D1A5D00091D2291091D329EF
:10141400083050E0104081F548E02AEF39E28D01B0
:101424000F948B0BE8EC31D00062008300810062E2
:1014340000830F944706002311F414D11DC090E0DB
:1014440099BF0C91FD019BBF07FF0CC002850F7370
:1014540019F401E0078B01C0978B11D002E0068BD1
:1014640019D00AC006811781012B11F404D104C0DC
:1014740006D001E0068BC1D0E4E00D946501928BA7
:10148400938B948B958B0895E0ECF4E030E03BBFB4
:101494000081089556D0033011F45AD051C0FD0193
:1014A400D1D042855385648975898A01061B170B3F
:1014B40080EC99E2202F212B29F50789002311F4D0
:1014C400E8D03EC002891389040F151F4681578155
:1014D4000417150720F08AD011F085D041F400E0FC
:1014E4000093F929FC010BBF028F038F25C08AD01A
:1014F40042851385042F242F2F7319F421E0278BA1
:1015040001C0378B013420E0120710F000E410E032
:10151400FC01028F138FFD01408551856489758913
:10152400460F571FFC01448F558FFD01448955898F
:10153400400F511F448B558BFC01008D0D7F008F94
:101544009BCF0F945401A2EEB9E20091F8290895BB
:10155400A3D02ACFF6DF043011F4FADF43C0809120
:10156400D2299091D329FD016DD004881588428534
:1015740053858001080F191F4017510718F4CA0139
:1015840080199109AC012AEF39E200851185000D1B
:10159400111D0F948B0BFD0155D004891589080F7B
:1015A400191F048B158B04898034904031F435D095
:1015B400668177814617570750F00287138716D044
:1015C40021F011D011F44ED00DC055D00BC042857E
:1015D40053854017510729F409D0A9F304D099F38E
:1015E40011D00BD049CF64D000230895478550898A
:1015F40061894030530763070895FADE00890D7F3F
:10160400008B0895FD0130E03BBF0489158905D0A6
:10161400428B538B348B358B089542895389400F09
:10162400511F08950ED0008905FD08C00091F829C6
:10163400013009F420C0043009F416D00895009351
:10164400F829D6DE30E03BBF0895FBDF008D05FDB1
:1016540008C00091F829023009F41BC0033009F4D2
:1016640003D0089505E0EBDF018D0460018F01894B
:101674000460018B089503E00093F82900E00093CF
:10168400DA290093DB29B4DE0BBF008D0D7F008FB8
:10169400089504E0D4DFB2CFE2EEF9E2D3DF44856B
:1016A4005585668540305307630709F001D00895D6
:1016B400FA016CBF1994EBECE8DE02FF07C0F0936B
:1016C400CA040091D82906FDADDF21C0008101FFC5
:1016D40008C002E007D00091D02906FFF6CFB5DF9D
:1016E400F4CF7DCD0093CA040895ECECCEDE00FF68
:1016F40076CD01E07CDE00890F77008B008D0F77BB
:10170400008F01E0EFDF00890F7E008B74DE01E0C3
:101714000895BD01D801F90130E006C03BBF219115
:1017240039BF2D9341505040242F252BB9F7DB01AD
:10173400089540E099BF4D9399B70150104020405F
:101744003040402F412B422B432B99F708953BBF48
:1017540007913BB799BF0D9399B7415050406040F2
:101764007040042F052B062B072B89F7089508EDED
:10177400402E07E1502E02E0602EF201362D6BBEA2
:101784004791579167917691F201EC5FFF4F3F4F7C
:101794003BBFA791B7919691F201362DE95FFF4FB8
:1017A4003F4F3BBF079117913691F801012B032B53
:1017B40011F0CDDF03C08A019B01BBDF0AE0400EBC
:1017C40000E0501E601EA201662D4C3E574162404F
:1017D400A0F20895EA080000502100000000D6009D
:1017E4000000722000EC1702030000000002006EEB
:1017F4000101760101000800007A01018001010362
:10180400000000840101000000040000008C0101BC
:101814000000000000000000000000000075207FB0
:10182400209D209D20892093209D209D209D209DEA
:10183400209D209D209D209D209D209D209D200059
:101844000003000000000000000000000000000091
:101854000000000000000000000000000000000084
:101864000000000041544D454C004446552041546D
:10187400584D45474131323841315500040309047C
:101884006D0601760601770601CA06010000000014
:101894001201000200000040EB03ED2F03000102DF
:1018A400000109021200010100C032090400000015
:0E18B400FF0000000A212C213E211A214021B4
:0400000320000000D9
:00000001FF
